:1078000011E0A0E0B1E0EEEFFFE702C005900D92BD
:10781000A230B107D9F721E0A2E0B1E001C01D928A
:10782000A83DB207E1F7CDB7DEB76897DEBFCDBFA1
:10783000112414BE88E18093600089E28093600087
:1078400085E080938100219A8AE05BD38FEE84B932
:1078500080E88AB963E083E2D9D16FE584E2D6D1CA
:107860006BE381E2D3D16CE485E2D0D167E286E2BA
:10787000CDD12ED263E780E5C9D166E08DE3C6D1D4
:107880006FE38CE3C3D16EEF80E2C0D18FE097E26B
:107890000197F1F700C0000043E050E060E070E0C5
:1078A0008DEC91E07BD348E050E06BE171E085EC3A
:1078B00091E074D38091CE01809300018FEF80938B
:1078C000CF012091CD012093A5012093A4018093A5
:1078D000AA018093A60182E08093A7018091A8016C
:1078E000887083608093A8012F3FD1F130E040E0A1
:1078F00050E060E070E080E090E034504E41574549
:1079000067457F4F8F4F9F4F29013A014B015C0123
:10791000298B5A8A4B8B7C8A6D8B9E8A8F8BB88E73
:1079200085E0FE017196A0EDB1E001900D928A957F
:10793000E1F745E0BE016F5E7F4F8AE255D149868F
:107940005A866B867C868D869E86AF86B88A45E091
:10795000BE01675F7F4F8BE247D163E082E256D181
:1079600068E087E0BAD1811101C09CD11092A601D4
:107970008091CD018F3FF1F489838CEF8A8381EE72
:107980008B8388EA8C838D831E821F82188645E054
:10799000BE016F5F7F4F8BE227D164E083E09DD112
:1079A000882339F08AE891E0C7D2682F80E090E020
:1079B00014D36FD1A8958091A701877080658093BB
:1079C000A7018091A8018871846C8093A80188E048
:1079D000E5ECF1E0ABEAB1E001900D928A95E1F7B8
:1079E00081E091E09093B4018093B30161E080E085
:1079F00074D1811101C056D180918E0190918F0177
:107A0000892B09F580919001909191018A379A4DC7
:107A100081F680918A0190918B018130910569F402
:107A2000A12CB12C6FEFC501D8D2FFEFAF1ABF0A5E
:107A3000A11424E0B206B1F7BCCF029709F0B9CF88
:107A400060918C01B3CF48E050E06AE871E085ECCA
:107A500091E08FD2892B09F425D18FEF9FEF90937E
:107A6000CC018093CB0148E050E06BE171E085EC04
:107A700091E0A4D288E0EAE8F1E0A5ECB1E0019061
:107A80000D928A95E1F78091A701877080638093BA
:107A9000A7018091C5019091C6019093AC0180939C
:107AA000AB018091C7019091C8019093AE01809382
:107AB000AD01A090C901B090CA0110E101E0E5E07C
:107AC0007E2EF1E16F2E450181E0881A9108909297
:107AD000B0018092AF0163E082E0FFD0882309F417
:107AE00068CF46E050E06AE871E08BEA91E041D26D
:107AF000892B09F045C091E0A91A90EFB90A8A2DA7
:107B000082958077A82FB0E0AE5FBE4FE0E9F1E04C
:107B1000912F01900D929A95E1F7811130C074E098
:107B2000AA0CBB1C7A95E1F783E0F50187BFE895C5
:107B300007B600FCFDCF4091020180E090E0DC013F
:107B4000AE5FBE4FFC01EA0DFB1D11962C91119703
:107B500030E0322F2227240F311D090107BFE8959D
:107B6000112412964C9102968038910541F7F50147
:107B700077BEE89507B600FCFDCF67BEE8955401D7
:107B8000A114B10409F09FCFA8954FD0882309F420
:107B900010CF48E050E06BE171E085EC91E00ED24F
:107BA00008CF98E087FF02C02B9A01C02B982D9A2E
:107BB00023B1880F22952170822B2D98915091F737
:107BC00008951F93CF93DF93EB01142F5F98E9DFA4
:107BD0001C0F1C1721F08FEFE4DF8993FACF5F9A17
:107BE000DF91CF911F9108951F93CF93DF93EB0106
:107BF000142F5F98D6DF1C0F1C1719F08991D1DF65
:107C0000FBCF5F9ADF91CF911F910895CF93DF93C0
:107C10001F92CDB7DEB7698341E0BE016F5F7F4F32
:107C2000E3DF0F90DF91CF9108958091C90190918A
:107C3000CA0124E0880F991F2A95E1F7E0E0F0E0FF
:107C40002FEF3FEFE817F907D1F044912427422F97
:107C500042954227042E469546954025042E46958A
:107C600040254770022E232F469507944795302DC7
:107C7000242706944795302524273196E3CF81E0C9
:107C80004091CB015091CC012417350709F080E0D9
:107C90000895F999FECF88E18093600088E0809391
:107CA0006000FFCFC2DF882341F088E1809360004D
:107CB00010926000E0E0F0E00994EBDF40E060E06B
:107CC00070E082EE91CF40E060E070E081EE8CCF1A
:107CD000F5DFF9DF60E787E299CF6F927F928F92AD
:107CE0009F92AF92BF92CF92DF92EF92FF920F934B
:107CF0001F93CF93DF93CDB7DEB7AA97DEBFCDBF7B
:107D0000762E8093A90105E051E2652EE4EAF1E0C8
:107D1000DE011196862D01900D928A95E1F7FB8088
:107D20001C81169516951695195F2091CE012898FD
:107D30002AA7CEDF6EEF80E269DF2AA530E040E0BF
:107D400050E060E070E080E090E034504E415745F4
:107D500067457F4F8F4F9F4F2AA33BA34CA35DA343
:107D60006EA37FA388A799A745E0BE016E5D7F4FF4
:107D70008AE23ADF45E0BE016E5D7F4F80E334DF8B
:107D80008FEFF81202C080EB01C080EA412FBE01E4
:107D90006F5F7F4F29DF289A95E39A95F1F70000EE
:107DA000289840E060E070E08FEF0BDF8073C9F34C
:107DB00060E787E22BDF84FD86DF6FE080E226DF6D
:107DC00087DF8090D0019090D101A090D201B09037
:107DD000D301C090D401D090D501E090D601F090AD
:107DE000D7019401A501B601C701A0E099D029F0FF
:107DF00045E060ED71E08AE2F7DE289A44E1E42E86
:107E000034E6F32EA89541E060E070E087E1D9DE2A
:107E100080FD5EC041E060E070E080E6D2DE182FB9
:107E2000813210F04BDF10E0412F63E871E081E612
:107E3000C8DE60E787E2EADE1123E9F1809186017E
:107E400087708230C1F5909185018091CD019813A2
:107E500032C050918701852F8770833019F580914A
:107E600088018830F9F47091000140918401741305
:107E700003C081E08093820160918A01262F30E067
:107E80008091CF0190E001972817390724F4809161
:107E90008201882311F0741305C06F5F6093CF01D6
:107EA0004093CE018091A8018527877021F48091AD
:107EB0008801871559F0FA9409F0A4CFEA9409F0E3
:107EC0009FCF015009F022CF80E009C081E007C0B8
:107ED0008FEC97E00197F1F700C00000ECCFAA9675
:107EE000DEBFCDBFDF91CF911F910F91FF90EF903B
:107EF000DF90CF90BF90AF909F908F907F906F90CA
:107F0000089528E13EEF91E03093850020938400AE
:107F100096BBB09BFECF199AA8958150A9F70895FA
:107F20000024A7FD00942A17300540055005600580
:107F30007005800590050895FC0188279927E8942D
:107F400021912032E9F3293010F02E30C8F32B3282
:107F500039F02D3231F4689403C018D0820F911D8E
:107F6000219120532A30C8F31EF4909581959F4F9C
:107F70000895FB01DC0104C08D910190801921F46A
:107F800041505040C8F7881B990B08957AE0979F9D
:107F9000902D879F802D910D11240895DC01CB0138
:107FA000FC01F999FECF06C0F2BDE1BDF89A319609
:107FB00000B40D9241505040B8F70895DC01A40F71
:107FC000B51F4150504040F0CB01840F951F2E91BA
:107FD00005D041505040D8F70895262FF999FECF8B
:107FE00092BD81BDF89A019700B4021639F01FBA0C
:0E7FF00020BD0FB6F894FA9AF99A0FBE0895C4
:027FFE00FF0082
:040000030000780081
:00000001FF
